:020000040800F2
:1000000000090020B1010008A123000859230008BD
:10001000812300085923000879230008B301000850
:10002000B3010008B3010008B30100083D34000823
:10003000B3010008B3010008B3010008B3010008D0
:10004000B3010008B3010008B3010008B3010008C0
:10005000B3010008B301000899410008C14100083C
:10006000E94100081142000839420008B3010008C4
:10007000B3010008B3010008B3010008B301000890
:10008000B3010008B3010008B30100080D23000804
:100090003923000849230008B30100086142000821
:1000A000B3010008B3010008B3010008B301000860
:1000B00035430008B3010008B3010008B30100088C
:1000C000B3010008B3010008B3010008B301000840
:1000D000B3010008B3010008B3010008B301000830
:1000E000C5420008B3010008B3010008B3010008CD
:1000F000B3010008B3010008B3010008B301000810
:10010000B3010008B3010008B3010008B3010008FF
:10011000B3010008B3010008B3010008B3010008EF
:10012000B3010008B3010008B3010008B3010008DF
:10013000B3010008B3010008B3010008B3010008CF
:10014000B3010008B3010008B3010008B3010008BF
:10015000B3010008B3010008B3010008B3010008AF
:10016000B3010008B3010008B3010008B30100089F
:10017000B3010008B3010008B3010008B30100088F
:10018000B3010008B3010008B3010008B30100087F
:10019000B3010008B3010008B3010008B30100086F
:1001A000150F000800000000000000000000000023
:1001B00002E000F000F8FEE772B6374880F30888E6
:1001C000364880F3098836483649086040F2000016
:1001D000CCF200004EF63471CEF200010860BFF39D
:1001E0004F8FBFF36F8F40F20000C0F2F0004EF669
:1001F0008851CEF200010860BFF34F8FBFF36F8FBD
:100200004FF00000E1EE100A4EF63C71CEF2000114
:100210000860062080F31488BFF36F8F03F0D6FDCB
:1002200003F058FE4FF055301F491B4A91423CBF26
:1002300041F8040BFAE71D49184A91423CBF41F8C6
:10024000040BFAE71A491B4A1B4B9A423EBF51F86E
:10025000040B42F8040BF8E700201849184A9142B1
:100260003CBF41F8040BFAE703F0B4FD03F086FE4F
:10027000144C154DAC4203DA54F8041B8847F9E7D7
:1002800000F042F8114C124DAC4203DA54F8041B52
:100290008847F9E703F09CBD000900200011002009
:1002A0000000000808ED00E0000100200009002027
:1002B00038450008001100207C110020801100202A
:1002C000043B0020A0010008A4010008A4010008CC
:1002D000A40100082DE9F04F2DED108AC1F80CD0D3
:1002E000C3689D46BDEC108ABDE8F08F002383F300
:1002F00011882846A047002003F010FAFEE703F01B
:1003000099F900DFFEE70000F8B500F015FE03F0F4
:10031000FFFC074603F050FD0646C0BB274B9F423B
:1003200035D001339F4235D0254B27F0FF029A424A
:1003300033D1F8B200F036FC354642F2107400F0CA
:1003400037FC08B10024254601F0E8F848B3032043
:1003500000F03AF80024254636B11A4B9F4203D0EC
:1003600003F022FD00242546002003F0DBFC0DB144
:1003700000F040F800F050FC02F01AF80546ACB965
:1003800000F092FC4FF47A7003F0CEF9F7E73546AF
:100390000024D4E704460125D1E705464FF47A74DA
:1003A000CDE7B4F57A7F08BF0125D5E702F000F864
:1003B000431BA342E4D900F01DF8DDE7010007B0BC
:1003C000000008B0263A09B0084B187003280CD872
:1003D000DFE800F008050208022000F007BE022056
:1003E00000F0FEBD024B00225A60704780110020D1
:1003F0008411002010B501F091F830B1234B032295
:100400001A70234B00225A6010BD224B224A1C4610
:1004100019680131F8D004339342F9D16268A242DD
:10042000F2D31E4B9B6803F1006303F520439A420D
:10043000EAD203F08BFC03F09DFC002000F096FD57
:100440000220FFF7C1FF164B9A6D00229A65996F43
:100450009A67996FD96DDA65D96FDA67D96F196EB6
:100460001A66D3F88010C3F88020D3F8803072B6B3
:100470004FF0E0233021C3F8084DD4E9003281F376
:1004800011889D4683F308881047BDE7801100203E
:100490008411002000A0000820A000080011002006
:1004A00000100240094A136849F2690099B21B0C16
:1004B00000FB01331360064B186844F2506182B2AE
:1004C000000C01FB0200186080B27047141100207C
:1004D0001011002010B500211022044600F0A0FDEC
:1004E000034B03CB206061601868A06010BD00BFA3
:1004F0009075FF1FF0B5ADF5517D6EAC4FF4C47231
:1005000007460D462046002100F08AFD01F050FF0D
:10051000244B4FF47A72B0FBF2F0186093E80700B6
:10052000022384E807000DF5ED702382FFF7D2FF68
:100530004BF214631C49238407A803F097FF1C2384
:1005400084F832310DF2EB226B440DF1340C1E466F
:1005500003CE664510605160334602F10802F6D1C1
:10056000306810600FAE31460122204600F0A4FD35
:1005700000230393AB7E029305F11903019380B22C
:100580000123CDE904600093E97E04A3D3E90023AD
:10059000384602F023FB0DF5517DF0BD9E6AC42163
:1005A000818A46EE8C1100207C4400082DE9F04140
:1005B0002C4C237ADAB080460D465BBB27A928462F
:1005C00000F0A0FE0746002842D19DF89D60C82E8D
:1005D0003ED801464FF4A662204600F021FD4FF4BC
:1005E0008073C4F8F8314FF40073C4F80C334FF43F
:1005F0004073C4F8203432460DF19E0104F1090025
:1006000000F0FCFC26449DF89C30777223720BB9F5
:10061000EB7E23728122002106AC27A800F000FDAA
:100620000122214627A800F0B3FE00230393AB7EEE
:10063000029305F1190380B201932823CDE9044008
:100640000093E97E05A3D3E90023404602F0C6FAF1
:100650005AB0BDE8F08100BFAFF30080264172724E
:10066000DF25D7B7D4210020F0B5254E4FF48A7589
:1006700005FB0065F1B096F8D83085F8DC30002431
:10068000D822214685F8E8403AA800F0C9FC06F1D6
:10069000090000F0BDFCD5F8E4308DF8F000C2B2DE
:1006A00006AF06F109010DF1F100CDE93A3400F091
:1006B000A5FC394601223AA800F0A0FE80B2CDE99F
:1006C000047008230127CDE9023706F1D80301930E
:1006D00030230093317A0B4807A3D3E9002302F0BB
:1006E0007DFAA04206DD01F063FEC5F8E000384661
:1006F00071B0F0BD2046FBE778F6339F93CACD8DED
:10070000D4210020A42100202DE9F0411D4D1E4ED2
:100710001E4F86B0284602F08DFA034658B30024D7
:10072000CDE90344ADF81440027B8DF8142099689C
:100730004068029403AA03C21B68DFF8548043F0A8
:100740000043029301F036FE821941F10003009448
:1007500002A9384601F0CAF8A04205DD284602F099
:100760006DFA88F80040D5E798F80030072B05D8D7
:10077000013388F8003006B0BDE8F081014802F08E
:100780005DFAF8E7A421002040420F001027002066
:100790000927002070B50D4614461E4602F07AF96E
:1007A00050B9022E10D1012C0ED112A3D3E900238F
:1007B000C5E90023012007E0282C10D005D8012C22
:1007C00009D0052C0FD0002070BD302CFBD10BA31D
:1007D000D3E90023ECE70BA3D3E90023E8E70BA35D
:1007E000D3E90023E4E70BA3D3E90023E0E700BF4C
:1007F000AFF30080401DA12026812A0B78F6339F9D
:1008000093CACD8D9E6AC421818A46EE26417272BA
:10081000DF25D7B7F017304A39059E5638B505465B
:100820000E4C0021013500F0C3FBA4F82C55B4F8A0
:100830002C0500F0A5FB78B1B4F82C0500F0B0FB56
:10084000014648B9B4F82C0500F0B2FBB4F82C35D9
:100850000133A4F82C35EAE738BD00BFD4210020CD
:1008600010B50A4B0A4A1A6003F5805393F87020BA
:100870003AB9DC6E2CB1204600F0CEFE204601F0E5
:100880000BF8BDE81040034800F0C6BE102700205A
:10089000D8440008683700202DE9F04F8FB000AF32
:1008A00005460C4602F0F6F800284BD1237E022BB9
:1008B0001BD1E38A012B18D101F07AFD0646FFF720
:1008C000F1FD03464FF4C870DFF8D482B3FBF0F2B9
:1008D00006F5167602FB103316FA83F3C8F80030DB
:1008E000E37E33B9A74B00221A703C37BD46BDE802
:1008F000F08F07F12401204600F0B8FC0028F4D165
:1009000007F11400FFF7E6FD97F8264007F1140100
:10091000224607F1270003F077FD0028E2D10F2CD3
:1009200008D8984B1C70D8F80030A3F51673C8F897
:100930000030DAE797F824100029D6D0284602F0D4
:10094000A1F8D2E7E38A282B33D010D8012B2BD083
:10095000052BCAD1BFF34F8F8B498C4BCA6802F469
:10096000E0621343CB60BFF34F8F00BFFDE7302B36
:10097000BBD1874EE17E327A9142B6D1607E31465C
:10098000002291F8DC50854200F0AD800132042A4B
:1009900001F58A71F5D1326840F6B831FA328A42EF
:1009A00094BF32603160A0E721462846FFF7A2FDE0
:1009B0009BE721462846FFF7F9FD96E7B2F8EC5091
:1009C0007B6005F103094FEA99094FEA8902D11DBD
:1009D000C908A8EBC1039D46EB460021584600F02C
:1009E0001FFB04F1EE012A463144584600F006FB95
:1009F0007B6813B9012000F0B9FA96F8D20000F034
:100A0000BFFA044630B9307200F0DAFA204600F03E
:100A1000ADFAB0E0D6F8D4203AB996F8D200B6F8DC
:100A20002C25824201D8FFF7F9FED6F8D4202A44BB
:100A3000944208D296F8D200B6F82C2501308242B2
:100A400001D8FFF7EBFE70685FFA89F2594600F0B3
:100A5000EFFA08B9C54679E0726896F8D2002A44E0
:100A60007260D6F8D42005EB0209C6F8D49000F0E5
:100A700087FA814509D396F8D220D6F8D4000132FE
:100A8000001B86F8D220C6F8D400FF2D0FD8002412
:100A9000347200F095FA204600F068FA00F03EFD4E
:100AA0003C4B188108B9FFF7A5FCC5461DE7BB689C
:100AB00096F8D9000AFB0362FB68D2F8E41082F8CA
:100AC000E83001F58061C2F8E030C2F8E410FFF7C9
:100AD000CBFDFFF719FE96F8D920013202F0030290
:100AE00086F8D920B6E74FF48A7A0AFB02F505F1B9
:100AF000EA013144204600F0B5FCF86000287FF49C
:100B0000F4AE3544012285F8E82001F051FCD5F817
:100B1000E020D6ED007ADFED206A801A192838BF70
:100B2000192040F6B832904228BF1046B8EE677AD6
:100B300007EE900AF8EEE77A67EEA67ADFED176A1D
:100B4000E7EE267AFCEEE77AC6ED007A96F8D93021
:100B50007168BB600AFB03F4321992F8E8505DB18A
:100B6000D2F8E4308B42E8463FF428AF002182F807
:100B7000E810C2F8E010C5467368064A9B0A0133C4
:100B80001381B2E69D21002000ED00E00400FA058B
:100B9000D42100208C110020CDCCCC3D6666663F70
:100BA000A0210020014B1870704700BF9811002051
:100BB00038B54FF00054144B22689A4221D1607D21
:100BC000F0B1124B124918701248237D03724FF492
:100BD0008073C0F8F8314FF40073C0F80C3300256F
:100BE0004FF44073C0F82034C0F8E450C9220930F3
:100BF00000F004FAE0222946204600F011FA012014
:100C000038BD0020FCE700BF9AAD44C59811002014
:100C100016000020D421002037B500F07FFC194DCC
:100C2000194928810223012218486B7101F05AFAF0
:100C300000230193164B174900931748174B4FF4A5
:100C4000805201F0F7FE164B197811B1124801F0ED
:100C500019FF01F0ADFB0446FFF724FC4FF4C87305
:100C6000B0FBF3F202FB130304F5167010FA83F0E5
:100C70000C4B186003F0A0F808B10F232B8103B0D0
:100C800030BD00BF8C11002040420F001027002013
:100C9000950700089C110020A42100209908000855
:100CA00098110020A02100202DE9F04F2DED028B9E
:100CB00090A7D7E900670FF24429D9E90089884C49
:100CC00095B00DAD9FED848BFFF71EFDDFF834B2BC
:100CD00000230C93ADF83C300D936B6000230DF1B5
:100CE00025028DED008B4FF0010A09A958468DF8B9
:100CF00025308DF824A001F0A3F99DF824200023CD
:100D0000002A40F0AF80204601F0C4FE05460028CE
:100D100047D1DFF8F4B101F04BFBDBF8003098422B
:100D20003FD301F045FB0790FFF7BCFB079A4FF458
:100D3000C873B0FBF3F101FB130302F5167010FA50
:100D400083F0CBF80000DFF8C4B19BF800100791E6
:100D5000002914BF2B46534610A88DF83030FFF7FA
:100D6000B9FB0799C1F11002D2B2062A10AB28BF15
:100D7000062219440DF13100079200F03FF9079A5D
:100D80000CAB0393182302930132564BD2B2CDE938
:100D900000A304923B463246204601F0C1FE8BF888
:100DA000005001F005FB504A504D1368C31AB3F5CB
:100DB0007A7F32D3106001F0FDFA02460B462046DE
:100DC00001F046FF204601F065FE30B32B7ADFF8D4
:100DD00040A1002B14BF032302238AF8053001F041
:100DE000E7FA0DF1400B4FF47A730122B0FBF3F0F8
:100DF0005946CAF80000504600F010FA1823029332
:100E00003B4B019380B240F25513CDE903B0009300
:100E100042464B46204601F083FE2B7AB3B101F0E7
:100E2000C7FA4FF0000A83464FF48A7295F8D9004A
:100E3000504400F0030002FB005393F8E81000292F
:100E400034D00AF1010ABAF1040FEFD1C82002F040
:100E50006BFC2B7A002B7FF434AF15B0BDEC028B0A
:100E6000BDE8F08F4FF0904110A84A6982F002026D
:100E70004A611946102200F0D3F80DF126030AAAA0
:100E80000CA9584600F038FE95E8030011AB83E842
:100E900003009DF83C308DF84C300C9B109310A94A
:100EA000DDE90A23204602F0A7F817E7D3F8E0109F
:100EB00049B12B68FA2B38BFFA23ABEB010105339C
:100EC000B1EB430FBDD3FFF7CFFB4FF48A7200287D
:100ED000B7D1BBE7AFF300800000000000000000C6
:100EE000A42100209C21002004270020D4210020E0
:100EF00008270020401DA12026812A0BF1C6A7C18A
:100F0000D068080F10270020A02100209D2100207C
:100F10008C11002008B5054800F08CFEBDE80840A3
:100F2000034A0449002003F04BBA00BF10270020F9
:100F3000303800206108000870B502F091FD094EBC
:100F4000094D3080002428683388834208D902F094
:100F500083FD2B6804440133B4F5204F2B60F2D39A
:100F600070BD00BF24380020F837002002F02ABEF0
:100F700000F10060920000F5204002F0ADBD0000DD
:100F8000054B1A68054B1B889B1A834202D91044F3
:100F900002F062BD00207047F8370020243800209E
:100FA000024B1B68184402F05DBD00BFF8370020FB
:100FB000024B1B68184402F067BD00BFF8370020E1
:100FC000064991F8243033B10023086A81F82430AF
:100FD0000822FFF7CDBF0120704700BFFC3700207B
:100FE000022804BF4FF0904398617047022802BF67
:100FF0004FF090434FF400329A61704710B50023D0
:10100000934203D0CC5CC4540133F9E710BD000017
:1010100003460246D01A12F9011B0029FAD1704783
:1010200002440346934202D003F8011BFAE77047DB
:101030002DE9F8431F4D144695F8242007468846AD
:1010400052BBDFF870909CB395F824302BB9202266
:10105000FF2148462F62FFF7E3FF95F82400C0F117
:101060000802A24228BF2246D6B24146920005EBB2
:101070008000FFF7C3FF95F82430A41B1E44F6B28E
:10108000082E17449044E4B285F82460DBD1FFF7C2
:1010900097FF0028D7D108E02B6A03EB8203834235
:1010A000CFD0FFF78DFF0028CBD10020BDE8F8831B
:1010B0000120FBE7FC3700202DE9F3470D460446ED
:1010C00000219046284640F27912FFF7A9FF2346F7
:1010D00020220021284601F031FF231D0222202179
:1010E000284601F02BFF631D03222221284601F030
:1010F00025FFA31D03222521284601F01FFF04F12F
:10110000080310222821284601F018FF04F11003DB
:1011100008223821284601F011FF04F111030822AA
:101120004021284601F00AFF04F112030822482159
:10113000284601F003FF04F1140320225021284621
:1011400001F0FCFE04F1180340227021284601F052
:10115000F5FE04F120030822B021284601F0EEFE3E
:1011600004F121030822B821284601F0E7FE04F12A
:101170002207C0263B46314608222846083601F0A1
:10118000DDFEB6F5A07F07F10107F3D194F8323008
:101190008DF8073031460DF107030822284601F08B
:1011A000CDFE002604F1330A9DF807304FEAC60948
:1011B0009E4209F5A47720D394F83231502B28BFF2
:1011C00050238DF80730B8F1000F08D139460DF1E2
:1011D00007030722284601F0B1FE09F24F17002647
:1011E00004F233149DF807309E4207EBC6010DD37D
:1011F0000731C80802B0BDE8F0870AEB06030822F1
:101200003946284601F09AFE0136CDE7A319082297
:10121000284601F093FE0136E4E7000013B50446CA
:101220000846002101602346C0F8031020220190E7
:1012300001F084FE0198231D0222202101F07EFE90
:101240000198631D0322222101F078FE0198A31D5D
:101250000322252101F072FE019804F108031022F7
:10126000282101F06BFE072002B010BDF7B5047F06
:1012700005460E462CB1838A122B02D9012003B0F9
:10128000F0BD0023194607220096284601F01AFDFA
:10129000731C0093012200230721284601F012FD50
:1012A000D4B9B31C0093052223460821284601F037
:1012B00009FD0D24B378102BE0D83746B278BB1B5C
:1012C000934210D32B7FA88A0734E408B3B9844231
:1012D00094BF00200120D2E7AB8ADB00083BDB088B
:1012E000B3700824E6E7FB1C009321460023082284
:1012F000284601F0E7FC08340137DFE7201A18BF61
:101300000120BCE7F7B5047F05460E462CB1838A61
:10131000CA2B02D9012003B0F0BD00231946009664
:101320000822284601F0CEFC731CD4B90822009391
:1013300011462346284601F0C5FC10247378C82BBB
:10134000E8D8012372785F1C013B934210D32B7FB6
:10135000A88A0734E408B3B9844294BF002001206E
:10136000D9E7AB8ADB00083BDB0873700824E5E7AC
:10137000F3190093214600230822284601F0A2FC1D
:1013800008343B46DEE7201A18BF0120C3E70000FF
:10139000F7B50D4604460021164628468122FFF780
:1013A0003FFE234608220021284601F0C7FD94F99C
:1013B00001206378002AB8BF7F238DF807309EB9DB
:1013C0000DF1070307220821284601F0B7FD0F277A
:1013D000002602349DF807309E4207EBC60105D374
:1013E0000731C80803B0F0BD0827F1E7A3190822A8
:1013F000284601F0A3FD0136ECE70000F7B50E46E4
:101400000546002114463046CE22FFF709FE2B4642
:1014100028220021304601F091FD2B7AC82B28BFED
:10142000C8238DF807308CB90DF107030822282155
:10143000304601F083FD30242F469DF807207B1BAA
:10144000934205D3E01DC00803B0F0BD2824F3E7A4
:1014500007F1090321460822304601F06FFD0834E8
:101460000137EAE7F7B5047F05460E4634B1838AB3
:10147000B3F5827F02D9012003B0F0BD00960123AD
:1014800010220021284601F01DFCDCB9B31C00939A
:10149000092223461021284601F014FC19247388E0
:1014A000B3F5807FE7D837467288BB1B934210D3D1
:1014B0002B7FA88A0734E408B3B9844294BF002084
:1014C0000120D9E7AB8ADB00103BDB0873801024D6
:1014D000E5E73B1D0093214600230822284601F042
:1014E000F1FB08340137DFE7201A18BF0120C3E7FA
:1014F00030B5094D0A4491420DD011F8013B5840D6
:10150000082340F30004013B2C4013F0FF0384EA5E
:101510005000F6D1EFE730BD2083B8EDF7B5384A7B
:10152000106851686B4603C36A463649364808233B
:1015300002F07AFF0446002833D10A25334A1068A6
:1015400051686B4603C36A4631492F48082302F0AD
:101550006BFF0446002849D00369B3F5583F45D8CE
:10156000B0F8661041F2B64291423FD1294A024496
:1015700002F15C018B4239D35C3B234900209E1A67
:10158000FFF7B6FF3246074604F164010020FFF77B
:10159000AFFFA3689F4229D1E368984208BF0025A6
:1015A00024E00369B3F5583F27D8418B41F2B64296
:1015B000914220D1174A024402F110018B4218D304
:1015C000103B114900209D1AFFF792FF2A4606465C
:1015D00004F118010020FFF78BFFA3689E4202D19F
:1015E000E368984201D00D25A8E70025284603B0FE
:1015F000F0BD1025A2E70C25A0E70B259EE700BF54
:101600009C440008DC5F030000A00008A54400081B
:10161000905F03000860FFF710B5037C044613B920
:10162000006802F0E9FE204610BD00000023BFF371
:101630005B8FC360BFF35B8FBFF35B8F8360BFF3D0
:101640005B8F7047BFF35B8F0068BFF35B8F7047A2
:1016500070B505460C30FFF7F5FF05F108060446A6
:101660003046FFF7EFFFA04206D930466D68FFF71E
:10167000E9FF2544281A70BD3046FFF7E3FF201A22
:10168000F9E7000070B50546406898B105F108001B
:10169000FFF7D8FF05F10C0604463046FFF7D2FFEE
:1016A0008442304694BF6D680025FFF7CBFF013CB4
:1016B0002C44201A70BD000038B50C460546FFF7D3
:1016C000C7FFA04210D305F10800FFF7BBFF044499
:1016D0006868B4FBF0F100FB1144BFF35B8F01209D
:1016E000AC60BFF35B8F38BD0020FCE72DE9F04113
:1016F000144607460D46FFF7C5FF844228BF04463F
:10170000D4B1B84658F80C6B4046FFF79BFF304405
:10171000286040467E68FFF795FF331A9C4203D845
:101720006C600120BDE8F0816B60A41B3B68AB607E
:101730002044E8600220F5E72046F3E738B50C4680
:101740000546FFF79FFFA04210D305F10C00FFF7FD
:1017500079FF04446868B4FBF0F100FB1144BFF367
:101760005B8F0120EC60BFF35B8F38BD0020FCE78E
:101770002DE9FF41884669460746FFF7B7FF6C46EB
:1017800006B204EBC6060025B44209D062682068A0
:1017900008EB0501FFF732FC636808341D44F3E7EA
:1017A00029463846FFF7CAFF284604B0BDE8F08155
:1017B000F8B505460C300F46FFF744FF05F1080663
:1017C00004463046FFF73EFFA042304688BF6C68B3
:1017D000FFF738FF201A386020B130462C68FFF739
:1017E00031FF2044F8BD000073B5144606460D468F
:1017F000FFF72EFF844228BF04460190DCB101A907
:101800003046FFF7D5FF019B33B93268C5E9023393
:10181000C5E9002401200CE09C4238BF01942860F7
:10182000019868608442F5D93368AB60241AEC6093
:10183000022002B070BD2046FBE700002DE9FF4109
:101840000F466946FFF7D0FF6C4600B204EBC005B7
:101850000026AC4209D0D4F8048054F8081BB8190B
:101860004246FFF7CBFB4644F3E7304604B0BDE801
:10187000F081000038B50546FFF7E0FF0446014659
:101880002846FFF719FF204638BD00000121884295
:1018900038BF084602F09ABD08B102F0ADBD7047EE
:1018A00010B4026854681A4623465DF8044B184782
:1018B00000207047002070477047000000207047EC
:1018C0000E20704700F5805090F8D800C0F340001B
:1018D0007047000000F5805090F9E000704700006C
:1018E00000F58050C0F8DC1001207047F7B50C6897
:1018F000BDF8207014F0005473D10D7B082D70D802
:10190000302585F31188456AAE6876010CD4AC6841
:10191000240108D4AC6814F0805460D184F3118899
:10192000204603B0F0BD01240E6804F1180C002E0F
:10193000B8BFF6004FEA0C1CB4BF46F004067605AB
:1019400045F80C600E680FFA84FC16F0804F18BF43
:1019500005EB0C1E05EB0C1C1EBFDEF8806146F08B
:101960000206CEF880610E7BCCF8846105EB04158D
:101970008E68C5F88C614E68C5F88861DCF88051C6
:1019800045F00105CCF8805141F2780500EB441C8C
:10199000660105EB4414AC440444CCE900230D4635
:1019A000083401F10C0C55F804EB44F804EB6545E0
:1019B000F9D12D882580841904F5805407F003059A
:1019C00094F8946026F00B06354384F89450002474
:1019D00084F31188009700F035FD0120A1E702246F
:1019E000A2E74FF0FF309CE713B500F5805401915A
:1019F000E06EFFF747FE1F280AD90199E06E20220A
:101A0000FFF7B6FEA0F120035842584102B010BDC6
:101A10000020FBE708B5302383F3118800F58050E0
:101A2000C06EFFF703FE002383F3118808BD00009A
:101A300000220260828142608260704710B50022FD
:101A40000023C0E900230023044603810C30FFF784
:101A5000EFFF204610BD0000F0B5054600F58050B0
:101A60000C4690F8D83013F0040FC3F3800108BF80
:101A7000114661F3820380F8D83005EB441303F577
:101A80008453103389B01B79D8074FEA44162FD5F9
:101A900082B319072ED46846FFF7D0FF05EB441335
:101AA00003F5845303AA03F108071868596814461C
:101AB00003C40833BB422246F7D1186820609B88D4
:101AC000A380DDE90E23CDE900230123ADF8083022
:101AD0002B6869461B6C28469847354405F58455A4
:101AE00010352B791A075CBF43F008032B7101E016
:101AF000002AF2D109B0F0BD2DE9F0479A4688B02E
:101B0000074688469146302383F3118807F58054B1
:101B10006846FFF793FFE06EFFF79AFD1F282AD96A
:101B2000E06E20226946FFF7A5FE202823D103ADF1
:101B3000444605AB2E4603CE9E422060616035468A
:101B400004F10804F6D130682060B388A380DDE991
:101B50000023C9E90023BDF80830AAF800300023AB
:101B600083F3118853464A464146384608B0BDE8DB
:101B7000F04700F02BBC002080F3118808B0BDE8CE
:101B8000F08700002DE9F84F182204460F46043074
:101B90000021FFF745FA2046234B40F8283BFFF78A
:101BA00047FF04F13800FFF749FF04F1580804F536
:101BB00082554646183530462036FFF73FFFAE4285
:101BC000F9D104F580554FF480534FF00009C5E971
:101BD0001739C5F858800123EE6604F5875804F5D7
:101BE0008456C5F8649085F8683085F870301836EA
:101BF00008F118084FF0000A4FF0000B46E908AB57
:101C0000A6F11800FFF714FF203646F8289C464539
:101C1000F4D185F8E07017B1044800F0C3FB044B21
:101C200063622046BDE8F88FD8440008B04400083D
:101C30000064004010B5044B197804464A1C1A7021
:101C4000FFF7A0FF204610BD2C3800202DE9F047FB
:101C5000002950D0294B2A4FB7FBF1F599428CBF90
:101C60000A231123581EB5FBF3FC03FB1C53C4B21B
:101C70002BB102280346F5D80020BDE8F0870CF10F
:101C8000FF36B6F5806FF7D2C4EBC40E0EF1030336
:101C90004FEAE309C3F3C703A4EB030809F1010A00
:101CA0004FF47A755FFA88F009FB05555AFA88F8FF
:101CB000B5FBF8F5B5F5617FC1BF0EF1FF33C3F396
:101CC000C703E01AC0B25C1C50FA84F40CFB04F4A5
:101CD000B7FBF4F4A142CFD1013BDBB20F2BCBD841
:101CE0000138C0B20728C7D8002110711680917042
:101CF000D3700120C1E70846BFE700BF3F420F0095
:101D000000B4C40470B505460E464FF47A746B6A8D
:101D10005B6803F00103B34207D04FF47A7001F01F
:101D200003FD013CF3D1204670BD0120FCE700001B
:101D300070B5426A936913F0700F17D000230C4DF1
:101D4000936141F2900400EB4312224411794E0753
:101D500009D5890707D5416A55F823608E60117946
:101D600041F0040111710133032BECD170BD00BFB0
:101D7000C444000873B51D46436A16469A68D207E4
:101D8000044609D59A6801219960C2F34002CDE961
:101D900000650021FFF760FE636A9A68D1050BD5E4
:101DA0009A684FF480719960C2F34022CDE90065D2
:101DB00001212046FFF750FE636A9A68D2030BD5D3
:101DC0009A684FF480319960C2F34042CDE90065D2
:101DD00002212046FFF740FE04F58053D3F8DC00D3
:101DE00010B103681B699847204602B0BDE87040F7
:101DF000FFF79EBFF8B50446466A002977D106F181
:101E00000C073868800775D006EB01153868D5F8DF
:101E1000B00110F0040FD5F8B0011ABFC00840F0AF
:101E20000040400DA062D5F8B0C11CF0020F1CBFED
:101E300040F08040A062D5F8B40106EB011100F03B
:101E40000F0084F83400D1F8B80184F82C00D1F8E0
:101E5000B801000A84F82D00D1F8B801000C84F80C
:101E60002E00D1F8B801000E84F82F00D1F8BC0183
:101E700084F83000D1F8BC01000A84F83100D1F8B0
:101E8000BC01000C84F83200D1F8BC11090E84F8B2
:101E900033103821396004F1440004F1280104F1C1
:101EA000340551F8046B40F8046BA942F9D1098854
:101EB0000180C4E90E2321460023A4F8403051F8E4
:101EC000383B20461B6C984704F5805393F8D82084
:101ED000D3F8DC0042F0040283F8D82010B1036884
:101EE0001B6998472046BDE8F840FFF721BF06F17F
:101EF000100786E7F8BD000010B5044600F05AFA56
:101F000002460B4652EA030102D0013A63F1000394
:101F10000449086820B12146BDE81040FFF76ABFB8
:101F200010BD00BF28380020F0B5302181F31188A2
:101F3000DFF848E000F583511831002441F2900C9D
:101F400000EB441565442E7977070ED4F6060CD5C0
:101F5000D1E9007697429E4107D2466A5EF8247026
:101F6000B7602E7946F004062E710134032C01F17E
:101F70002001E5D1002383F31188F0BDC44400089B
:101F800008B5302383F31188FFF7D2FE002383F3D3
:101F9000118808BD2DE9F041436A0446986800F0B5
:101FA000E050B0F1E05F0E4622D0F8B1302383F369
:101FB0001188002504F5845741F2900804EB45137D
:101FC00043441B791A0706D50135032D07F1200775
:101FD000F4D1012007E05B07F6D43946304600F023
:101FE00083FA0028F0D1002383F31188BDE8F08143
:101FF0000120FBE708B5302383F3118800F58050FA
:10200000C06EFFF725FB002383F3118843090CBF43
:102010000120002008BD0000F8B51D460023137004
:102020000F4606461446FFF7E5FF80F001003870C2
:1020300025B129463046FFF7ADFF2070F8BD0000FE
:102040002DE9B8410C4615461F46804600F0B2F90E
:102050000B462178024609B9287850B14046FFF76F
:1020600063FFFFF78DFF3B462A462146FFF7D4FF6B
:102070000120BDE8B881000070B5302686F31188D4
:10208000174B9A6D42F000729A659A6B42F000729B
:102090009A639A6B22F000729A63002383F311888B
:1020A00000F5805494F8D83013F0010516D1A9B189
:1020B00086F311880321132001F032FA0321142042
:1020C00001F02EFA0321152001F02AFA94F8D830F5
:1020D00043F0010384F8D83085F3118870BD00BF48
:1020E000001002402DE9F04700F5805588B095F8C2
:1020F000E030012B04468846164600F28280824F6B
:1021000057F823200AB947F82300D7F800A0C4F8ED
:102110001C8084F82060BAF1000F64D095F8E0309C
:10212000012B70D001212046FFF7A6FF302383F357
:102130001188626A136823F002031360626A1368ED
:1021400043F001031360636A00275F6187F311881E
:1021500001212046FFF7D6FD002800F09580E86EAB
:10216000FFF764FA04F58359BA4609F118092022E9
:1021700000216846FEF754FF02A8FFF759FCCDF88E
:1021800018A06A4609EB07030DF1180E9446BCE847
:102190000300F44518605960624603F10803F5D165
:1021A000DCF80000186020379CF804201A71602FBA
:1021B000DDD195F8D8306FF38203002785F8D83049
:1021C0006A4641462046ADF80070ADF802708DF8C1
:1021D0000470FFF73BFD636A48BB4FF400421A608E
:1021E00008B0BDE8F08741F2E800FFF74FFB8146F9
:1021F00010B15146FFF7C6FCC7F80090B9F1000FC7
:102200008CD10020ECE7386803681B6B98470146C7
:10221000002887D13868FFF72FFF386803683246F7
:102220005B684146984700287FF47CAFE9E761226C
:102230001A609DF802309DF803201B06120402F478
:10224000702203F040731343BDF80020C2F309026B
:1022500013439DF804201205022E02F4E0020CBF85
:102260004FF0004100211343626A0B43D361636A5C
:1022700013225A61626A136823F00103136039461E
:102280002046FFF73FFD08B9636AA6E795F8E030FE
:1022900093BB616AD1F8002242F00102C1F800222A
:1022A000616AD1F8002222F47C5222F00E02C1F8B9
:1022B0000022616AD1F8002242F46062C1F8002273
:1022C000626AC2F81432626AC2F80432626A41F683
:1022D000FF71C2F80C12626AC2F84032626AC2F838
:1022E0004432636A0122C3F81C22626AD2F80032C7
:1022F00023F00103C2F8003295F8D83043F002030E
:1023000085F8D8306CE700BF2838002008B500F009
:1023100051F850EA0103024602D0421E61F1000169
:10232000044B186810B10B46FFF724FDBDE80840C8
:1023300001F0B8B82838002008B50020FFF7DCFD10
:10234000BDE8084001F0AEB808B50120FFF7D4FDA4
:10235000BDE8084001F0A6B800B59BB0EFF30981D5
:1023600068226846FEF74AFEEFF30583014B9B6B3C
:10237000FEE700BF00ED00E008B5FFF7EDFF00004D
:1023800000B59BB0EFF3098168226846FEF736FE80
:10239000EFF30583014B5B6BFEE700BF00ED00E050
:1023A000FEE700000FB408B5029801F06DF9FEE7F2
:1023B00001F048BC01F02ABC0139C9B202299EBF14
:1023C00000EBC1000023C0E901337047F8B51B885A
:1023D0005B0705460E4615D4044600F11807BC42BB
:1023E00010D0636853B12B682846DB6B9847A3680D
:1023F000C1B23246606898470834F0E7A368002B02
:10240000F1D1F9E70120F8BD73B56C4684E8060008
:10241000014600224E68D5B26EB98E685EB900EBF7
:10242000C200021D94E80300013582E803001D701C
:10243000012002B070BD0132032A01F10801E9D187
:102440000020F6E72DE9F04F89B00446BDF848704A
:102450000E46054600F118084FF0000907F0040782
:102460004FF0000A4FF0000BA84538D06B680BB94D
:10247000AB684BB157B923682046DB6B9847AB6814
:10248000C1B23246686898470835EDE7B9F1000FE8
:10249000FAD1CDE900ABADF80890334603AA06F1B6
:1024A000080E186859689446ACE803000833734571
:1024B0006246F6D11868CCF800009B88ACF804306E
:1024C000FFF778FF0423ADF808302368CDE9000159
:1024D0001B6C6946204698474FF00109D4E701205C
:1024E00009B0BDE8F08F000030B503680968DD0F62
:1024F000B5EBD17F23F0604421F060424FEAD17008
:102500000BD0002BB8BFA40C0029B8BF920C94428A
:1025100002D034BF0120002030BD944205D1C1F368
:102520008070C3F380738342F6D194422CBF0020A5
:102530000120F1E72DE9F041456A15B94162BDE896
:10254000F0814B6823F06047C3F38A464FEAD37E9D
:10255000C3F3807816EA230638BF3E46AC462B46C6
:102560005A68BEEBD27F22F060440AD0002A18DA03
:10257000A40CB44217D19D420FD10D60DEE7134683
:10258000EEE7A74207D102F08044C2F380724245D1
:102590000BD054B1EFE708D2EDE7CCF800100B6098
:1025A000CDE7B44201D0B442E5D81A689C46002A6F
:1025B000E5D11960C3E700002DE9F047089D01F05F
:1025C00007044FEAD508224405F0070500EBD100C7
:1025D0004FF47F49944201D1BDE8F08704F007072A
:1025E00005F0070A57453E4638BF5646C6F108066D
:1025F000111B8E4228BF0E46E10808EBD50E415C48
:1026000013F80EC0B94029FA06F721FA0AF1FFB211
:102610008CEA010147FA0AF739408CEA010C03F809
:102620000EC034443544D5E780EA0120082341F246
:10263000210201B24000002980B203F1FF33B8BF8C
:10264000504013F0FF03F4D17047000038B50C463A
:102650008D18A54200D138BD14F8011BFFF7E4FF27
:10266000F7E7000042684AB11368436043898189F3
:1026700001339BB29942438138BF83811046704732
:1026800070B588B0202204460D4668460021FEF74A
:10269000C7FC20460495FFF7E5FF024658B16B469C
:1026A000054608AE1C4603CCB44228606960234648
:1026B00005F10805F6D1104608B070BD082817D9F5
:1026C00009280CD00A280CD00B280CD00C280CD0D0
:1026D0000D280CD00E2814BF4020302070470C204D
:1026E0007047102070471420704718207047202032
:1026F00070470000082817D90C280CD910280CD9CD
:1027000014280CD918280CD920280CD930288CBFB3
:102710000F200E207047092070470A2070470B20B9
:1027200070470C2070470D20704700002DE9F843DA
:10273000078C072F04461ED9D0E9029800254FF6D2
:10274000FF73C5F12006A5F1200029FA05F108FA6A
:1027500006F628FA00F031430143C9B21846FFF7E4
:1027600063FF0835402D0346EBD1E1693A46BDE8E9
:10277000F843FFF76BBF4FF6FF70BDE8F88300002A
:1027800010B54B6823B9CA8A63F30902CA8210BD27
:1027900004691A681C600361C38A013BC3824A60F2
:1027A000EFE700002DE9F84F1D46CB8A0F46C3F333
:1027B00009010529814692460B4630D00020AAB275
:1027C00007F11A049EB2042E1FFA80F80FD8904524
:1027D00003F1010306D3FB8A0A4462F30903FB8277
:1027E00001201AE01AF80060E6540130EAE790454B
:1027F000F1D2A1F1050B1C237C68BBFBF3F203FBB8
:1028000012BB1FFA8BF6002C45D14846FFF72AFF72
:10281000044638B978606FF00200BDE8F88F4FF0D9
:102820000008E6E7002606607860ADB24FF0000BC6
:10283000454510D90AEB0803221D13F8011B9155D9
:10284000B1B208F101081B291FFA88F82BD04545C1
:1028500006F10106F1D8FB8AC3F30902154465F3BA
:102860000903BCE7013292B21C462368002BF9D160
:102870006B1F0B441C21B3FBF1F301339BB29A4253
:10288000D3D2BBF1000FD0D14846FFF7EBFE20B901
:10289000C4F800B0BFE70122E7E7C0F800B05E4629
:1028A00020600446C1E74545D5D94846FFF7DAFE22
:1028B00008B92060AFE7C0F800B0002620600446E9
:1028C000B6E700002DE9F04F2DED028B1C4683B0DA
:1028D0005B69019207468846002B00F0A780238C95
:1028E0002BB1E269002A00F0A180072B35D807F14F
:1028F0000C00FFF7B7FE054638B96FF00205284611
:1029000003B0BDEC028BBDE8F08F14220021FEF76E
:1029100087FB228CE16905F10800FEF76FFB208C34
:10292000013080B2FFF7E6FEFFF7C8FE013880B243
:102930002084013028746369228C1B782A4403F0B8
:102940001F0363F03F0348F000411372384669608B
:102950002946FFF7EFFD0125D1E702339BB207229D
:10296000C18A0633B3FBF2F3828A521A9BB292B247
:102970009342C2D800F10C034FF0000908EE103A60
:102980004FF0800A4E464D4618EE100AFFF76AFED9
:1029900083460028B1D014220021FEF741FB002E0F
:1029A0003AD1019BABF8083002220BF1080E1FFA56
:1029B00082FC0CF10100BCF1060F218C80B201D821
:1029C0008E422BD3FFF796FEFFF778FE62691278EE
:1029D000013802F01F028E4208BF4FF0400A42EA5F
:1029E00049121BFA80F14AEA020A013048F000421B
:1029F00081F808A08BF81000CBF80420594638461F
:102A0000FFF798FD238C0135B3422DB289F00109FF
:102A10004FF0000AB8D172E70022C6E7E169895D8C
:102A20000EF802100136B6B20132C0E76FF00105B0
:102A300065E70000F8B515460E4630220021044631
:102A40001F46FEF7EDFA069B6360B5F5001F079B76
:102A5000A76034BF6A094FF6FF72A36297B2E661BE
:102A600004F1100000239A4206D800230360A782D5
:102A7000E3822383E360F8BD0660013330462036ED
:102A8000F1E7000003781BB94BB2002BC8BF0170FF
:102A90007047000000787047F8B50C46C9690746D2
:102AA00011B9238C002B37D1257E1F2D34D83878CF
:102AB00028BB228C072A2CD8268A36F003032BD178
:102AC0004FF6FF70FFF7C2FD20F001003102400415
:102AD00041EA0561400C41EA40254FF6FF7223466A
:102AE00029463846FFF7EEFE002807DD62691378B5
:102AF0000133DBB21F2B88BF00231370F8BD218A7E
:102B00002D0645EA012505432046FFF70FFE024644
:102B1000E5E76FF00300F1E76FF00100EEE700007A
:102B200070B58AB0044616460021282268461D4624
:102B3000FEF776FABDF83830ADF810300F9B0593EC
:102B40009DF840308DF81830119B07936946BDF809
:102B50004830ADF820302046CDE90265FFF79CFFF4
:102B60000AB070BD2DE9F041D36905460C46164602
:102B70000BB9138C5BBB377E1F2F28D895F80080CC
:102B8000B8F1000F26D03046FFF7D0FD3378210290
:102B900041EAC33141EA0801338A41EA076141EA67
:102BA00003410246334641F080012846FFF78AFE82
:102BB00000280ADD3378012B07D1726913780133BD
:102BC000DBB21F2B88BF00231370BDE8F0816FF0CC
:102BD0000100FAE76FF00300F7E70000F0B58BB0F3
:102BE00004460D4617460021282268461E46FEF779
:102BF00017FA9DF84C305A1E534253418DF800305D
:102C00009DF84030ADF81030119B05939DF8483089
:102C10008DF81830149B07936A46BDF85430ADF810
:102C2000203029462046CDE90276FFF79BFF0BB006
:102C3000F0BD0000406A00B104307047436A1A6872
:102C4000426202691A600361C38A013BC382704712
:102C50002DE9F041D0F82080194E14461D4641461A
:102C6000002709B9BDE8F081D1E90223A21A65EB7A
:102C70000303964277EB03031ED2036A8B420DD106
:102C8000FFF77EFD036A1B68036203690B60C38A5A
:102C90000161016A013BC3828846E2E7FFF770FDEC
:102CA0000B68C8F8003003690B60C38A0161013BFF
:102CB000C382D8F80010D4E788460968D1E700BF7E
:102CC00080841E002DE9F04F8BB00D46DDF850904A
:102CD00014469B468046002800F01981B9F1000F88
:102CE00000F01581531E3F2B00F21181012A03D100
:102CF000BBF1000F40F00B810023CDE90833B8F899
:102D00001430B5EBC30F4FEAC30703D300200BB059
:102D1000BDE8F08F2B199F42D8F80C303ABF7F1BCB
:102D2000FFB227461BB9D8F81030002B7AD0272DD8
:102D30004ED8C5F12806B7424FF000032CBFF6B2BB
:102D40003E4600932946D8F8080008AB3246FFF704
:102D500033FCA7EB060A35445FFA8AFAB8F8143058
:102D600003F10053053BDB000493D8F80C300393C8
:102D70002821039B13B1BAF1000F2CD1D8F8100011
:102D800040B1BAF1000F05D0009608AB5246691A5F
:102D9000FFF712FC38B2002FB8D066070AD00AAB92
:102DA00003EBD401624211F8083C02F00702134120
:102DB00001F8083C082C3CD9102C40F2B580202C9E
:102DC00040F2B780BBF1000F00F09C80082334E094
:102DD000BA460026C2E7049BE02B28BFE0230693F7
:102DE0000B44AB42059314D95A1B039800969245A5
:102DF00034BF5246D2B2691A08AB04300792FFF7CB
:102E0000DBFB079A1644AAEB020A1544F6B25FFAF6
:102E10008AFA049B069A05999B1A0493039B1B68E4
:102E20000393A6E70093D8F8080008AB3A46294672
:102E3000AEE7BBF1000F13D00123B4EBC30F6CD08E
:102E4000082C12D89DF82030621E23FA02F2D50712
:102E500006D54FF0FF3202FA04F423438DF82030F8
:102E60009DF8203089F8003051E7102C12D8BDF8B9
:102E70002030621E23FA02F2D10706D54FF0FF324E
:102E800002FA04F42343ADF82030BDF82030A9F84D
:102E900000303CE7202C0FD80899631E21FA03F379
:102EA000DA0705D54FF0FF3202FA04F40C43089418
:102EB000089BC9F800302AE7402C2BD0DDE90865D3
:102EC000611EC4F12102A4F1210326FA01F105FAE1
:102ED00002F225FA03F311431943CB0712D501225D
:102EE000A4F12003C4F1200102FA03F322FA01F154
:102EF000A240524243EA010363EB430332432B43B4
:102F0000CDE90823DDE90823C9E90023FFE66FF0D6
:102F10000100FCE66FF00800F9E6082CA0D9102C9F
:102F2000B3D9202CEED8C3E7BBF1000FADD00223FC
:102F300083E7BBF1000FBBD004237EE730B5012A45
:102F4000144638BF0124402C85B028BF40240025FA
:102F5000012ACDE9025518D81B788DF8083063078F
:102F60000AD004AB03EBD405624215F8083C02F02A
:102F70000702934005F8083C0091034622460021D1
:102F800002A8FFF719FB05B030BD082AE4D9102AC2
:102F900003D81B88ADF80830E1E7202A8DBFD3E9BC
:102FA00000231B680293CDE90223D8E710B5CB6854
:102FB0001BB98B600B618B8210BD04691A681C60A1
:102FC0000361C38A013BC382CA60F0E703064CBFBA
:102FD000C0F3C0300220704708B50246FFF7F6FF85
:102FE000022806D15306C2F30F2001D100F00300DE
:102FF00008BDC2F30740FBE72DE9F04F93B0CDE9E0
:1030000003230A6804461046FFF7E0FF022814BFB6
:10301000C2F306260026002A0D46824680F2F7817A
:1030200012F0C04940F0F381097B002900F0EF81E4
:10303000022803D02378B34240F0EC81C2F304634A
:103040000693104602F07F030593FFF7C5FF059B2B
:1030500029444FEA834848EA0A4848EA4668CE7855
:1030600000230022CDE90823F309834648EA00083B
:10307000029367D0059B009302466768534608A9F0
:103080002046B847002800F0C881276A4FB941465A
:1030900004F10C00FFF7F4FA074690B96FF0020054
:1030A00054E03B6998450DD03F68002FF9D1414667
:1030B00004F10C00FFF7E4FA07460028EED0236A7B
:1030C0003B60276297F817C006F01F08CCF3840C0A
:1030D000ACEB08001FFA80FE0028B8BF0EF12000FC
:1030E000A8EB0C031FFA83FED7E90221B8BF00B298
:1030F000002B0793BEBF0EF120031BB2079352EAC9
:10310000010338D0039BDFF824E39A1A049B4FF0A5
:10311000000C63EB010196457CEB01032BD36B7B29
:1031200097F81AE0734519D1029B002B78D001283B
:1031300021DC7868F8B9DFF8F0C2944570EB010340
:1031400016D337E0276A27B96FF00C0013B0BDE83B
:10315000F08F3B699845B5D03F68F4E7B24890429C
:103160007CEB010301D30020F0E7029B002BFAD097
:10317000079B0F2B17DCFA7DB30002F0030203F06C
:103180007C031343FB7539462046FFF7F9FA6B7B46
:10319000BB76029B3BB9FB7DC3F38402013262F331
:1031A0008603FB75D0E76A7BBB7E9A42DBD1029B2C
:1031B000002B35D0B309022B32D0039BBB60049B9C
:1031C000FB60142200210DA8FDF72AFF039B0A9340
:1031D000049B0B932B1D0C932B7BADF83EB0013B56
:1031E000DBB2ADF83C30069B8DF84230059B8DF884
:1031F000433094F82C308DF840A083F001038DF813
:1032000044308DF84180A3680AA920469847FB7D89
:10321000C3F38403013303F01F039B02FB82A2E785
:10322000FB7DC6F34012B2EBD31F40F0F980C3F32D
:103230008403434540F0FC80029A2B7BB609002AA8
:1032400052D016F0010661D1032B40F2F480039BAB
:10325000BB60049BFB60FB8A66F30903FB822B7B4C
:10326000AE1D033BDBB23246394604F10C00FFF7DA
:1032700099FA00280CDA39462046FFF781FAFB7DDF
:10328000C3F38403013303F01F039B02FB8205E7B2
:10329000DDE90884AB883B834FF6FF73C9F120005A
:1032A000A9F1200228FA09F104FA00F0014324FAF6
:1032B00002F211431846C9B2FFF7B6F909F108093D
:1032C000B9F1400F0346E9D1B8822A7B033AD2B262
:1032D0003146FFF7BBF9FB7DB882DA43C2F3C01277
:1032E00062F3C713FB753EE786B92E1D013BDBB2C7
:1032F0003246394604F10C00FFF754FA0028BADBD5
:103300002A7BB88A013AD2B23146E2E7F98AC1F3A0
:103310000901013B0429DAB25BD8281D002307F11B
:103320001B069A4208D910F801CB06F801C00131FA
:1033300001330529DBB2F4D103990A9104990B9169
:10334000934207F11B010C9138BF043379680D914A
:1033500034BF55FA83F300230E93FB8AADF83EB0D9
:10336000C3F309031A44069B8DF84230059B8DF880
:10337000433094F82C30ADF83C2083F001038DF8F5
:10338000443000238DF840A08DF841807B602A7B7B
:10339000B88A013A291DFFF759F93B8BB88283425D
:1033A00003D1A3680AA92046984720460AA9FFF737
:1033B000FDFDFB7DBA8AC3F38403013303F01F03D1
:1033C0009B02FB823B8B9A420CBF00206FF01000E7
:1033D000BCE67B68002BAFD0052001E01C303346F3
:1033E0001E68002EFAD1091A081D2E1D184401EB83
:1033F000090CBCF11B0F5FFA89F39DD89A429BD947
:1034000016F8013B00F8013B09F10109EFE76FF005
:1034100009009BE66FF00A0098E66FF00B0095E656
:103420006FF00D0092E600BF40420F0080841E0046
:103430006FF00E008AE66FF00F0087E6EFF3098366
:1034400005494A6B22F001024A63683383F3098815
:10345000002383F31188704700EF00E0302080F3F1
:10346000118862B60C4B0D4AD96821F4E061090459
:10347000090C0A43DA60D3F8FC20094942F0807253
:10348000C3F8FC200A6842F001020A602022DA77C1
:1034900083F82200704700BF00ED00E00003FA054A
:1034A000001000E010B5302383F311880E4B5B68E9
:1034B00013F4006314D0F1EE103AEFF30984683C82
:1034C0004FF08073E361094BDB6B236684F309885B
:1034D00000F0A4F810B1064BA36110BD054BFBE74B
:1034E00083F31188F9E700BF00ED00E000EF00E092
:1034F000FF020008020300084FF0E0230022586892
:103500004FF0FF31930003F1604303F56143013253
:103510009042C3F88010C3F88011F3D270470000C6
:1035200000F1604303F561430901C9B283F8001358
:10353000012200F01F039A4043099B0003F16043FE
:1035400003F56143C3F880211A60704700230375B7
:10355000826803691B6899689142FBD25A680360CC
:1035600042601060586070470023037582680369E9
:103570001B6899689142FBD85A68036042601060EA
:103580005860704708B50846302383F311880B7DD7
:10359000032B05D0042B0DD02BB983F3118808BD64
:1035A0008B6900221A604FF0FF338361FFF7CEFF73
:1035B0000023F2E7D1E9003213605A60F3E700001C
:1035C000FFF7C4BF054BD9680875186802681A6010
:1035D000536001220275D860FCF77CBE38380020A9
:1035E00030B50C4BDD684B1C87B004460FD02B4622
:1035F000094A684600F02AF92046FFF7E3FF009BDE
:1036000013B1684600F02CF9A86907B030BDFFF788
:10361000D9FFF9E73838002085350008044B1A68CF
:10362000DB6890689B68984294BF00200120704737
:1036300038380020084B10B51C68D86822681A601A
:10364000536001222275DC60FFF78EFF01462046A1
:10365000BDE81040FCF73EBE3838002038B5074CB6
:1036600007490848012300252370656000F0EAFB44
:103670000223237085F3118838BD00BF603A002013
:10368000204500083838002008B572B6044B18658C
:1036900000F0ACFA00F058FB024B03221A70FEE770
:1036A00038380020603A002000F010B98B60022307
:1036B00008618B82084670478368A3F1840243F84F
:1036C000142C026943F8442C426943F8402C094AFF
:1036D00043F8242CC26843F8182C022203F80C2C5F
:1036E000002203F80B2C044A43F8102CA3F120000D
:1036F000704700BFED0200083838002008B5FFF71A
:10370000DBFFBDE80840FFF75BBF0000024BDB6852
:1037100098610F20FFF756BF38380020302383F31D
:103720001188FFF7F3BF000008B50146302383F38B
:1037300011880820FFF754FF002383F3118808BD88
:1037400010B503689C68A2420CD85C688A600B6064
:103750004C602160596099688A1A9A604FF0FF3373
:10376000836010BD1B68121BECE700000A2938BFFC
:103770000A2170B504460D460A26601900F05CFB6C
:1037800000F048FB041BA54203D8751C2E460446D6
:10379000F3E70A2E04D9BDE87040012000F092BB87
:1037A00070BD0000F8B5144B0D46D96103F110014E
:1037B00041600A2A1969826038BF0A2201604860A4
:1037C0001861A818144600F029FB0A2700F022FB14
:1037D000431BA342064606D37C1C281900F02CFB91
:1037E00027463546F2E70A2F04D9BDE8F840012004
:1037F00000F068BBF8BD00BF38380020F8B50646B9
:103800000D4600F007FB0F4A134653F8107F9F4206
:1038100006D12A4601463046BDE8F840FFF7C2BF50
:10382000D169BB68441A2C1928BF2C46A34202D97F
:103830002946FFF79BFF224631460348BDE8F84082
:10384000FFF77EBF383800204838002010B4C0E9A8
:10385000032300235DF8044B4361FFF7CFBF000053
:1038600010B5194C236998420DD0D0E90032816817
:1038700013605A609A680A449A60002303604FF00C
:10388000FF33A36110BD2346026843F8102F536035
:103890000022026022699A4203D1BDE8104000F084
:1038A000C5BA936881680B44936000F0B3FA22694B
:1038B000E1699268441AA242E4D91144BDE810407B
:1038C000091AFFF753BF00BF383800202DE9F04731
:1038D000DFF8BC8008F110072C4ED8F8105000F02B
:1038E00099FAD8F81C40AA68031B9A423ED814449F
:1038F000D5E900324FF00009C8F81C4013605A6047
:10390000C5F80090D8F81030B34201D100F08EFA1B
:1039100089F31188D5E9033128469847302383F38A
:1039200011886B69002BD8D000F074FA6A69A0EB9B
:1039300004094A4582460DD2022000F0C3FA002253
:10394000D8F81030B34208D151462846BDE8F047B8
:10395000FFF728BF121A2244F2E712EB090938BF19
:103960004A4629463846FFF7EBFEB5E7D8F810304F
:10397000B34208D01444211AC8F81C00A960BDE85D
:10398000F047FFF7F3BEBDE8F08700BF48380020DE
:103990003838002038B500F03DFA054AD2E908452C
:1039A000031B181945F10001C2E9080138BD00BF29
:1039B0003838002000207047FEE700007047000004
:1039C0004FF0FF3070470000BFF34F8F024A13697A
:1039D000DB03FCD4704700BF0020024008B5094B50
:1039E0001B7873B9FFF7F0FF074B5A69002ABFBF76
:1039F000064A9A6002F188329A601A6822F480625C
:103A00001A6008BD783A0020002002402301674573
:103A100008B50B4B1B7893B9FFF7D6FF094B5A69D2
:103A200042F000425A611A6842F480521A601A68E1
:103A300022F480521A601A6842F480621A6008BD4B
:103A4000783A0020002002407F289ABF00F580309D
:103A5000C0020020704700004FF400607047000073
:103A6000802070477F2808B50BD8FFF7EDFF00F5E1
:103A700000630268013204D104308342F9D101208D
:103A800008BD0020FCE700007F2810B504461FD8C1
:103A9000FFF79AFFFFF7A2FF0E4BF3221A610222F3
:103AA0005A615A6942EAC0025A615A6942F4803244
:103AB0005A61FFF789FF4FF40061FFF7C5FF00F07F
:103AC0003FF9FFF7A5FF2046BDE81040FFF7CABF4A
:103AD000002010BD002002402DE9F84340EA020317
:103AE00013F00703144606D0304B40F282321A60BE
:103AF0000020BDE8F88385182D4A95420CD92B4A41
:103B000040F287311160F3E7031D1B684A68934256
:103B100008D1083C08300831072C14D902680B681A
:103B20009A42F1D0FFF75AFFFFF74EFF214E0831BE
:103B30004FF001084FF00009012CA1F1080706D849
:103B4000FFF766FF01E0002CECD10120D1E7C6F8B9
:103B50001480054651F8083C45F8043B51F8043CF4
:103B60004360FFF731FF336943F001033361C6F867
:103B70001490026851F8083C9A420CD00B4B40F26A
:103B8000AF321A600C4B18600C4B1C600C4B1F6062
:103B9000FFF73EFFACE72D6851F8043C9D4201F170
:103BA0000801EBD1083C0830C6E700BF743A00209A
:103BB0000000040800200240683A0020703A00200B
:103BC0006C3A0020084908B50B7828B11BB9FFF7FB
:103BD00005FF01230B7008BD002BFCD0BDE8084099
:103BE0000870FFF715BF00BF783A002002484FF475
:103BF0007F4100F0A7B800BF000100200846114631
:103C000000F0E4BB084600F0F7BB000038B5EFF366
:103C100011859DB9EFF30584C4F30804302334B152
:103C200083F31188FFF7B6FE85F3118838BD83F35F
:103C30001188FFF7AFFE84F3118838BDBDE8384026
:103C4000FFF7A8BE38B5FFF7E1FF114C114AC008D5
:103C500040EA4170A0FB025EC908A0FB040C1CEB0B
:103C6000050CA1FB04404FF000035B41A1FB0212D5
:103C70001CEB040C43EB000011EB0E0142F10002BF
:103C8000411842F10000090941EA007038BD00BF47
:103C9000CFF753E3A59BC42010B50244064BD2B224
:103CA000904200D110BD441C00B253F8200041F8EE
:103CB000040BE0B2F4E700BF50280040114B30B5D0
:103CC000D3F89040240409D4D3F89040C3F890402E
:103CD000D3F8904044F40044C3F890400A4C236861
:103CE00043F4807323600244084BD2B2904200D167
:103CF00030BD441C00B251F8045B43F82050E0B2E0
:103D0000F4E700BF0010024000700040502800405F
:103D100007B5012201A90020FFF7BEFF019803B0FB
:103D20005DF804FB13B50446FFF7F2FFA04205D08F
:103D3000012201A900200194FFF7C0FF02B010BDCD
:103D4000704700007047000070470000074B45F2C5
:103D500055521A6003225A6040F2FF729A604CF684
:103D6000CC421A60024B01221A70704700300040AA
:103D7000803A0020034B1B781BB1034B4AF6AA2262
:103D80001A607047803A002000300040054B1A68E6
:103D900032B902F1804202F50432D2F894201A605E
:103DA000704700BF7C3A0020024B4FF40002C3F87A
:103DB000942070470010024008B5FFF7E7FF024B60
:103DC0001868C0F3407008BD7C3A002070470000BE
:103DD000FEE700000A4B0B480B4A90420BD30B4BFB
:103DE000DA1C121AC11E22F003028B4238BF0022D5
:103DF0000021FDF715B953F8041B40F8041BECE74C
:103E0000B4450008043B0020043B0020043B002094
:103E100000F0C0B84FF08043586A70474FF08043BD
:103E2000002258631A610222DA6070474FF0804323
:103E30000022DA60704700004FF0804358637047FB
:103E4000FEE7000070B51B4B01630025044686B0F9
:103E5000586085620E46FFF701FB04F11003C4E9C8
:103E600004334FF0FF33C4E90635C4E90044A560CC
:103E7000E562FFF7CFFF2B460246C4E9082304F1B1
:103E800034010D4A256580232046FFF70FFC0123EE
:103E9000E0600A4A0375009272680192B268CDE947
:103EA0000223074B6846CDE90435FFF727FC06B02F
:103EB00070BD00BF603A00202C4500083145000865
:103EC000413E0008024AD36A1843D062704700BFDF
:103ED00038380020254B2648DA6A42F0070210B431
:103EE000DA62DA6A22F00702DA62DA6ADA6C42F03F
:103EF0000702DA64DA6E42F00702DA664FF09042A7
:103F0000DB6E4FF0AA31002353604FF41924916007
:103F1000D0604FF6FD70506113625462154C14600E
:103F2000154CC2F80434C2F80844C2F80C34C2F884
:103F3000140441F20400C2F82034C2F82434C2F858
:103F40000004C2F80438C2F808184FF6FF71C2F82E
:103F50000C38C2F81418C2F82038C2F82438C2F855
:103F600000385DF8044B00F055B800BF0010024067
:103F7000000001240400812AA69AAAAA08B500F02C
:103F800005FAFFF76BFBBDE80840FFF7FFBE000036
:103F9000704700000F4B9A6D42F001029A659A6FCC
:103FA00042F001029A670C4A9B6F936843F0010349
:103FB00093604FF080434F229A624FF0FF32DA62F3
:103FC00000229A615A63DA605A6001225A611A60CB
:103FD000704700BF00100240002004E04FF0804214
:103FE00008B51169D3680B40D9B2C9439B07116169
:103FF00007D5302383F31188FFF756FB002383F3A3
:10400000118808BD08B5FFF777FABDE8084000F051
:1040100099B900005A4B4FF0FF319A6A99629A6A37
:1040200000229A62986AD86A60F00700D862D86A5B
:1040300000F00700D862D86A186B1963186B1A630E
:10404000186B986B9963986B9A63986BD86BD9636C
:10405000D86BDA63D86B186C1964196C1A641A6C13
:10406000484A4FF4E06111601A6E474942F001027C
:104070001A66D3F8802022F00102C3F88020D3F81A
:1040800080209A6D42F080529A659A6F22F0805299
:104090009A679A6F4FF440720A604A6912F480621C
:1040A000FBD14A601A6822F0F00242F060021A6006
:1040B0001A6842F001021A601A689107FCD50022C2
:1040C0009A609A6812F00C02FBD1D3F8901011F4A8
:1040D000407F1EBF4FF48031C3F89010C3F890208A
:1040E00061221A601A689207FCD500229A609A68C9
:1040F00012F00C0FFBD169221A60D3F8942022F43D
:10410000706242F4C062C3F894201A6842F48032AC
:104110001A601A689003FCD5D3F8902022F003228D
:10412000C3F89020194ADA601A6842F080721A6067
:104130001A689101FCD5164A1A611A6842F0806229
:104140001A601A681201FCD500229A600D49114AC2
:10415000C3F888200A6822F0070242F004020A60CD
:104160000A6802F00702042AFAD19A6842F00302B0
:104170009A609A6802F00C020C2AFAD1704700BFCC
:1041800000100240002002400070004013140001A3
:10419000100C100055550134074A08B5536903F057
:1041A0000103536123B1054A13680BB15068984766
:1041B000BDE80840FFF776B900040140843A0020CA
:1041C000074A08B5536903F00203536123B1054A56
:1041D00093680BB1D0689847BDE80840FFF762B913
:1041E00000040140843A0020074A08B5536903F0EF
:1041F0000403536123B1054A13690BB15069984711
:10420000BDE80840FFF74EB900040140843A0020A1
:10421000074A08B5536903F00803536123B1054AFF
:1042200093690BB1D0699847BDE80840FFF73AB9E8
:1042300000040140843A0020074A08B5536903F09E
:104240001003536123B1054A136A0BB1506A9847B2
:10425000BDE80840FFF726B900040140843A002079
:10426000164B10B55C6904F478725A61A30604D544
:10427000134A936A0BB1D06A9847600604D5104A76
:10428000136B0BB1506B9847210604D50C4A936B06
:104290000BB1D06B9847E20504D5094A136C0BB1FA
:1042A000506C9847A30504D5054A936C0BB1D06CAC
:1042B0009847BDE81040FFF7F5B800BF0004014083
:1042C000843A0020194B10B55C6904F47C425A61B1
:1042D000620504D5164A136D0BB1506D984723053E
:1042E00004D5134A936D0BB1D06D9847E00404D503
:1042F0000F4A136E0BB1506E9847A10404D50C4AB7
:10430000936E0BB1D06E9847620404D5084A136FC0
:104310000BB1506F9847230404D5054A936F0BB136
:10432000D06F9847BDE81040FFF7BCB800040140CB
:10433000843A002008B5FFF751FEBDE80840FFF7BA
:10434000B1B80000062108B50846FFF7E9F80621D4
:104350000720FFF7E5F806210820FFF7E1F806211E
:104360000920FFF7DDF806210A20FFF7D9F806211A
:104370001720FFF7D5F806212820FFF7D1F8BDE870
:10438000084007211C20FFF7CBB8000008B5FFF755
:1043900039FE00F007F8FFF7FBFDBDE80840FFF726
:1043A00037BD00000023054A19460133102BC2E92E
:1043B000001102F10802F8D1704700BF843A0020D2
:1043C0000B460146184600F009B80000024B0A46A9
:1043D00001461868FFF712BC1811002010B5054CF3
:1043E00013462CB10A4601460220AFF3008010BDEF
:1043F0002046FCE700000000024B01461868FFF76A
:1044000001BC00BF1811002010B5013902449042D0
:1044100001D1002005E0037811F8014FA34201D03B
:10442000181B10BD0130F2E72DE9F041A3B1C91A04
:1044300017780144044603F1FF3C8C42204601D921
:10444000002009E00578BD4204F10104F5D10CEB30
:104450000405D618A54201D1BDE8F08115F8018DFB
:1044600016F801EDF045F5D0E7E70000034611F836
:10447000012B03F8012B002AF9D17047696E2E73C6
:1044800069657272616165726F73706163652E54E4
:104490007275654E617649430000000040A2E4F168
:1044A000646891060041A3E5F26569920700000087
:1044B0004261642043414E496661636520696E64D0
:1044C00065782E0080000000008000000000800061
:1044D0000000000000000000A1180008E52000080E
:1044E00041200008E1180008ED180008F91A00083A
:1044F000B1180008C1180008B5180008BD18000858
:10450000B9180008151A0008C51800080924000881
:10451000B9230008D5180008E91900086330000025
:104520001C45000890380020603A00206D61696EDB
:104530000069646C65000000B61400000000000013
:104540000060030000000000FE2A0100D204000009
:104550001C1100200000000000000000000000000E
:10456000000000000000000000000000000000004B
:10457000000000000000000000000000000000003B
:10458000000000000000000000000000000000002B
:10459000000000000000000000000000000000001B
:1045A000000000000000000000000000000000000B
:0445B0000000000007
:00000001FF
